:020000040000FA
:1000000007309F00003085000030860083160030E6
:100010008500CB3086001930990024309800831277
:1000200090309800A801A80B13281A081A081A087B
:10003000342003018C1E19282120A9002320292007
:1000400019281A08080099008316981C252883127D
:10005000080029088500291E0612291A0616A91E5D
:100060008612A91A861608000030232000302320AB
:10007000003023200030232000302320532048303C
:1000800023206F3023206C30232061302320203048
:100090002320613023206D302320693023206730F6
:0E00A00023206F3023200D3023200A30232828
:02400E00503F21
:00000001FF
